******************************************************************************
               TMS320C6x Linker PC v7.4.21                     
******************************************************************************
>> Linked Wed Jun 14 11:11:28 2017

OUTPUT FILE NAME:   <testUn.out>
ENTRY POINT SYMBOL: "_c_int00"  address: 00806020


MEMORY CONFIGURATION

         name            origin    length      used     unused   attr    fill
----------------------  --------  ---------  --------  --------  ----  --------
  VECTORS               00800000   00000200  00000000  00000200  RWIX
  LL2_RW_DATA           00800200   000bfe00  0000b8cc  000b4534  RWIX
  SL2                   0c000000   00100000  00000000  00100000  RWIX
  DDR3_CODE             80000000   01000000  00000000  01000000  RWIX
  DDR3_R_DATA           81000000   01000000  00000220  00fffde0  RWIX
  DDR3_RW_DATA          82000000   06000000  00000000  06000000  RWIX


SEGMENT ALLOCATION MAP

run origin  load origin   length   init length attrs members
----------  ----------- ---------- ----------- ----- -------
00800200    00800200    00006140   00006140    r-x
  00800200    00800200    00006140   00006140    r-x .text
00806340    00806340    00005000   00000000    rw-
  00806340    00806340    00004000   00000000    rw- .sysmem
  0080a340    0080a340    00001000   00000000    rw- .stack
0080b340    0080b340    000002b4   000002b4    r--
  0080b340    0080b340    000002b4   000002b4    r-- .const
0080b5f8    0080b5f8    00000290   00000000    rw-
  0080b5f8    0080b5f8    00000290   00000000    rw- .far
0080b888    0080b888    00000248   00000248    r--
  0080b888    0080b888    00000248   00000248    r-- .cinit
81000000    81000000    00000220   00000220    rw-
  81000000    81000000    00000220   00000220    rw- .fardata


SECTION ALLOCATION MAP

 output                                  attributes/
section   page    origin      length       input sections
--------  ----  ----------  ----------   ----------------
.text      0    00800200    00006140     
                  00800200    00004c60     bignum.obj (.text)
                  00804e60    00000280     rts6600_elf.lib : memory.obj (.text:free)
                  008050e0    00000240                     : imath64.obj (.text:__c6xabi_divull)
                  00805320    00000180                     : copy_decompress_rle.obj (.text:__TI_decompress_rle_core)
                  008054a0    00000180                     : memory.obj (.text:malloc)
                  00805620    00000100                     : autoinit.obj (.text:_auto_init_elf)
                  00805720    00000100                     : cpy_tbl.obj (.text:copy_in)
                  00805820    00000100     main.obj (.text)
                  00805920    000000e0     rts6600_elf.lib : copy_zero_init.obj (.text:decompress:ZI:__TI_zero_init)
                  00805a00    000000e0                     : memset.obj (.text:memset)
                  00805ae0    000000c0                     : divu.obj (.text:__divu)
                  00805ba0    000000c0                     : exit.obj (.text:exit)
                  00805c60    000000c0                     : tls.obj (.text:tls:init:__TI_tls_init)
                  00805d20    000000a0                     : memory.obj (.text:_minit)
                  00805dc0    000000a0                     : memcpy64.obj (.text:memcpy)
                  00805e60    000000a0                     : memory.obj (.text:minsert)
                  00805f00    000000a0                     : memory.obj (.text:mremove)
                  00805fa0    00000080                     : llshift.obj (.text:__c6xabi_llshl)
                  00806020    00000080                     : boot.obj (.text:_c_int00)
                  008060a0    00000080                     : memory.obj (.text:calloc)
                  00806120    00000060                     : cpp_init.obj (.text:__TI_cpp_init)
                  00806180    00000060                     : llshift.obj (.text:__c6xabi_llshru)
                  008061e0    00000060                     : imath64.obj (.text:_subcull)
                  00806240    00000040                     : strasg.obj (.text:__strasgi_64plus)
                  00806280    00000040                     : args_main.obj (.text:_args_main)
                  008062c0    00000020                     : _lock.obj (.text:_nop)
                  008062e0    00000020                     : exit.obj (.text:abort)
                  00806300    00000020                     : copy_decompress_none.obj (.text:decompress:none:__TI_decompress_none)
                  00806320    00000020                     : copy_decompress_rle.obj (.text:decompress:rle24:__TI_decompress_rle24)

.sysmem    0    00806340    00004000     UNINITIALIZED
                  00806340    00000008     rts6600_elf.lib : memory.obj (.sysmem)
                  00806348    00003ff8     --HOLE--

.stack     0    0080a340    00001000     UNINITIALIZED
                  0080a340    00000008     rts6600_elf.lib : boot.obj (.stack)
                  0080a348    00000ff8     --HOLE--

.const     0    0080b340    000002b4     
                  0080b340    000002a0     bignum.obj (.const:small_prime)
                  0080b5e0    00000014     bignum.obj (.const:.string)

.far       0    0080b5f8    00000290     UNINITIALIZED
                  0080b5f8    00000290     main.obj (.far)

.cinit     0    0080b888    00000248     
                  0080b888    00000220     (.cinit..fardata.load) [load image, compression = rle]
                  0080baa8    0000000c     (__TI_handler_table)
                  0080bab4    00000008     (.cinit..far.load) [load image, compression = zero_init]
                  0080babc    00000004     --HOLE-- [fill = 0]
                  0080bac0    00000010     (__TI_cinit_table)

.fardata   0    81000000    00000220     
                  81000000    00000100     main.obj (.fardata:N0)
                  81000100    00000100     main.obj (.fardata:T0)
                  81000200    0000000c     rts6600_elf.lib : exit.obj (.fardata)
                  8100020c    0000000c                     : memory.obj (.fardata)
                  81000218    00000008                     : _lock.obj (.fardata)


LINKER GENERATED COPY TABLES

__TI_cinit_table @ 0080bac0 records: 2, size/record: 8, table size: 16
	.fardata: load addr=0080b888, load size=00000220 bytes, run addr=81000000, run size=00000220 bytes, compression=rle
	.far: load addr=0080bab4, load size=00000008 bytes, run addr=0080b5f8, run size=00000290 bytes, compression=zero_init


LINKER GENERATED HANDLER TABLE

__TI_handler_table @ 0080baa8 records: 3, size/record: 4, table size: 12
	index: 0, handler: __TI_zero_init
	index: 1, handler: __TI_decompress_rle24
	index: 2, handler: __TI_decompress_none


GLOBAL SYMBOLS: SORTED ALPHABETICALLY BY Name 

address    name
--------   ----
008062e0   C$$EXIT
81000000   N0
81000100   T0
0080b5f8   T_out
0080bac0   __TI_CINIT_Base
0080bad0   __TI_CINIT_Limit
0080baa8   __TI_Handler_Table_Base
0080bab4   __TI_Handler_Table_Limit
UNDEFED    __TI_INITARRAY_Base
UNDEFED    __TI_INITARRAY_Limit
0080b340   __TI_STACK_END
00001000   __TI_STACK_SIZE
00000000   __TI_STATIC_BASE
00004000   __TI_SYSMEM_SIZE
UNDEFED    __TI_TLS_INIT_Base
UNDEFED    __TI_TLS_INIT_Limit
00000001   __TI_args_main
00806120   __TI_cpp_init
00806300   __TI_decompress_none
00806320   __TI_decompress_rle24
81000208   __TI_enable_exit_profile_output
ffffffff   __TI_pprof_out_hndl
ffffffff   __TI_prof_data_size
ffffffff   __TI_prof_data_start
00805c60   __TI_tls_init
00805920   __TI_zero_init
ffffffff   __binit__
00805ae0   __c6xabi_divu
008050e0   __c6xabi_divull
00805fa0   __c6xabi_llshl
00806180   __c6xabi_llshru
00806240   __c6xabi_strasgi_64plus
ffffffff   __c_args__
00805ae0   __divu
00806240   __strasgi_64plus
00806280   _args_main
00805620   _auto_init_elf
00806020   _c_int00
81000200   _cleanup_ptr
81000204   _dtors_ptr
81000218   _lock
00805d20   _minit
008062c0   _nop
0080a340   _stack
008061e0   _subcull
00806340   _sys_memory
8100021c   _unlock
008062e0   abort
ffffffff   binit
008060a0   calloc
00805720   copy_in
00805ba0   exit
00804e60   free
00805908   main
008054a0   malloc
00800b50   mbedtls_mpi_add_abs
00803088   mbedtls_mpi_add_int
00801e78   mbedtls_mpi_add_mpi
008002d4   mbedtls_mpi_bitlen
00800828   mbedtls_mpi_cmp_abs
008007f0   mbedtls_mpi_cmp_int
00800630   mbedtls_mpi_cmp_mpi
00800458   mbedtls_mpi_copy
00802580   mbedtls_mpi_div_int
00801f14   mbedtls_mpi_div_mpi
00803890   mbedtls_mpi_exp_mod
00803648   mbedtls_mpi_fill_random
00800368   mbedtls_mpi_free
00804408   mbedtls_mpi_gcd
00804b6c   mbedtls_mpi_gen_prime
00804b30   mbedtls_mpi_get_bit
008003c4   mbedtls_mpi_grow
00800330   mbedtls_mpi_init
0080462c   mbedtls_mpi_inv_mod
00804370   mbedtls_mpi_is_prime
0080352c   mbedtls_mpi_lsb
00800994   mbedtls_mpi_lset
0080054c   mbedtls_mpi_mod_int
00803464   mbedtls_mpi_mod_mpi
00801e54   mbedtls_mpi_mul_int
00801c64   mbedtls_mpi_mul_mpi
00803354   mbedtls_mpi_read_binary
008030c0   mbedtls_mpi_read_string
00802e94   mbedtls_mpi_safe_cond_assign
00802c78   mbedtls_mpi_safe_cond_swap
00802bd0   mbedtls_mpi_set_bit
008009f0   mbedtls_mpi_shift_l
00800f18   mbedtls_mpi_shift_r
00802ad4   mbedtls_mpi_shrink
008029b4   mbedtls_mpi_size
00800d64   mbedtls_mpi_sub_abs
00802aa0   mbedtls_mpi_sub_int
00800e80   mbedtls_mpi_sub_mpi
00802a60   mbedtls_mpi_swap
008029cc   mbedtls_mpi_write_binary
008026a8   mbedtls_mpi_write_string
00805dc0   memcpy
00805a00   memset
0080b788   sig_out


GLOBAL SYMBOLS: SORTED BY Symbol Address 

address    name
--------   ----
00000000   __TI_STATIC_BASE
00000001   __TI_args_main
00001000   __TI_STACK_SIZE
00004000   __TI_SYSMEM_SIZE
008002d4   mbedtls_mpi_bitlen
00800330   mbedtls_mpi_init
00800368   mbedtls_mpi_free
008003c4   mbedtls_mpi_grow
00800458   mbedtls_mpi_copy
0080054c   mbedtls_mpi_mod_int
00800630   mbedtls_mpi_cmp_mpi
008007f0   mbedtls_mpi_cmp_int
00800828   mbedtls_mpi_cmp_abs
00800994   mbedtls_mpi_lset
008009f0   mbedtls_mpi_shift_l
00800b50   mbedtls_mpi_add_abs
00800d64   mbedtls_mpi_sub_abs
00800e80   mbedtls_mpi_sub_mpi
00800f18   mbedtls_mpi_shift_r
00801c64   mbedtls_mpi_mul_mpi
00801e54   mbedtls_mpi_mul_int
00801e78   mbedtls_mpi_add_mpi
00801f14   mbedtls_mpi_div_mpi
00802580   mbedtls_mpi_div_int
008026a8   mbedtls_mpi_write_string
008029b4   mbedtls_mpi_size
008029cc   mbedtls_mpi_write_binary
00802a60   mbedtls_mpi_swap
00802aa0   mbedtls_mpi_sub_int
00802ad4   mbedtls_mpi_shrink
00802bd0   mbedtls_mpi_set_bit
00802c78   mbedtls_mpi_safe_cond_swap
00802e94   mbedtls_mpi_safe_cond_assign
00803088   mbedtls_mpi_add_int
008030c0   mbedtls_mpi_read_string
00803354   mbedtls_mpi_read_binary
00803464   mbedtls_mpi_mod_mpi
0080352c   mbedtls_mpi_lsb
00803648   mbedtls_mpi_fill_random
00803890   mbedtls_mpi_exp_mod
00804370   mbedtls_mpi_is_prime
00804408   mbedtls_mpi_gcd
0080462c   mbedtls_mpi_inv_mod
00804b30   mbedtls_mpi_get_bit
00804b6c   mbedtls_mpi_gen_prime
00804e60   free
008050e0   __c6xabi_divull
008054a0   malloc
00805620   _auto_init_elf
00805720   copy_in
00805908   main
00805920   __TI_zero_init
00805a00   memset
00805ae0   __c6xabi_divu
00805ae0   __divu
00805ba0   exit
00805c60   __TI_tls_init
00805d20   _minit
00805dc0   memcpy
00805fa0   __c6xabi_llshl
00806020   _c_int00
008060a0   calloc
00806120   __TI_cpp_init
00806180   __c6xabi_llshru
008061e0   _subcull
00806240   __c6xabi_strasgi_64plus
00806240   __strasgi_64plus
00806280   _args_main
008062c0   _nop
008062e0   C$$EXIT
008062e0   abort
00806300   __TI_decompress_none
00806320   __TI_decompress_rle24
00806340   _sys_memory
0080a340   _stack
0080b340   __TI_STACK_END
0080b5f8   T_out
0080b788   sig_out
0080baa8   __TI_Handler_Table_Base
0080bab4   __TI_Handler_Table_Limit
0080bac0   __TI_CINIT_Base
0080bad0   __TI_CINIT_Limit
81000000   N0
81000100   T0
81000200   _cleanup_ptr
81000204   _dtors_ptr
81000208   __TI_enable_exit_profile_output
81000218   _lock
8100021c   _unlock
ffffffff   __TI_pprof_out_hndl
ffffffff   __TI_prof_data_size
ffffffff   __TI_prof_data_start
ffffffff   __binit__
ffffffff   __c_args__
ffffffff   binit
UNDEFED    __TI_INITARRAY_Base
UNDEFED    __TI_INITARRAY_Limit
UNDEFED    __TI_TLS_INIT_Base
UNDEFED    __TI_TLS_INIT_Limit

[99 symbols]
